:1000000023C03DC03CC03BC03AC039C038C037C037
:1000100036C035C034C033C032C031C030C02FC04C
:100020002EC02DC02CC02BC02AC080C028C027C025
:1000300026C025C034C135C136C137C138C139C128
:100040003AC13BC13CC13DC111241FBECFEFD2E03C
:10005000DEBFCDBF12E0A0E0B1E0ECEBF0E102C00A
:1000600005900D92AA30B107D9F712E0AAE0B2E0EC
:1000700001C01D92AA39B107E1F77AD11DC8C0CFDE
:100080002AEF30E0E22FF32F3197F1F7A8958A9508
:10009000C9F708958436910518F422E030E002C0D3
:1000A00023E030E0C901089564E670E0BAD7CB01DF
:1000B000089564E670E0B5D76AE070E0B2D7CB018E
:1000C0000895EAE7F0E0808181608083808182602A
:1000D000808380818B7F8083ACE7B0E08C918064EB
:1000E0008C93808188608083808180688083808118
:1000F00080648083089580917A00806480937A0080
:1001000080917A0086FDFCCF2091780030917900B3
:10011000C90108958FEF8AB91BB8209A219A229AB3
:10012000269A289A299A2A9A2E9A08951F920F920F
:100130000FB60F9211242F933F938F93EF93FF935A
:1001400080910E022091780030917900E82FF0E044
:10015000EE0FFF1FEE5EFD4F318320838F5F809394
:100160000E02FF91EF918F913F912F910F900FBE53
:100170000F901F90189510920E022091120230914C
:100180001302C90146E0880F991F4A95E1F7820FD3
:10019000931F909399028093980226E096958795F5
:1001A0002A95E1F79093930280939202909397029D
:1001B000809396020895609196027091970280E074
:1001C00090E0C5D420E030E040E650E49DD320E04C
:1001D00030E040E251E4A3D2DED070939702609306
:1001E00096026431710540F480E090E0B0D426E6D8
:1001F00036E646EC5FE30AC06E31710570F480E0CC
:1002000090E0A5D423E333E343E95FE388D2C3D08E
:10021000709397026093960208956639710568F0AD
:1002200080E090E094D426EF38E24CE75FE377D2A9
:10023000B2D070939702609396020895209196022F
:1002400030919702C9016AE070E0EBD680930F020B
:10025000C9016AE070E0E5D6CB016AE070E0E1D662
:1002600080939402C90164E670E0DBD6CB016AE0BA
:1002700070E0D7D680931102C90168EE73E0D1D641
:10028000CB016AE070E0CDD6809395020895E82F07
:10029000F0E0EA30F105B0F4E65EFF4F09948CEF30
:1002A000089580E508958EE6089586E7089582ED25
:1002B000089586EB08958EEB089580E708958EEFFC
:1002C000089586EF0895289A299A2A9A2E9A6230DC
:1002D00061F0633018F4613069F405C0633039F0BF
:1002E000643041F406C0289805C0299803C02A98B4
:1002F00001C02E988BB98AEF90E021E0E82FF92F0A
:100300003197F1F7A8952A95C9F7289A299A2A9A38
:100310002E9A08951F9381E023C0123069F01330A4
:1003200018F41130B1F405C0133049F0143089F4D9
:100330000BC0809195020AC08091110207C0809184
:100340009402A5DF816003C080910F02A0DF80933B
:10035000100280911002612FB6DF809100018F5F43
:1003600080930001109100011530B8F21F9108959B
:10037000D1DEA7DE789480917A00806480937A0041
:1003800080910E02803429F410920E02F4DE13DF05
:1003900055DFC0DFF0CFEF92FF920F931F937B01E9
:1003A0008C0120E030E040E05FE455D388237CF00E
:1003B000C801B70120E030E040E05FE45ED176D3D1
:1003C0009B01AC01205030404040504805C0C8015E
:1003D000B7016CD39B01AC01B901CA011F910F9108
:1003E000FF90EF900895A0E0B0E0E8EFF1E02DC6B7
:1003F000DC012B01FA019C91923008F439C1EB0128
:100400008881823008F433C1943069F4843009F073
:100410002FC111969C9111978981981709F428C1D1
:10042000A1E0B1E025C1843009F421C18230A9F4F2
:10043000923009F01DC19A01AD0188E0EA010990EE
:10044000AE01E90109929E018150C1F7E201898163
:1004500011969C918923818308C1923009F407C1C8
:1004600012962D903C901397EB018A819B811496F4
:10047000AD90BD90CD90DC901797EC80FD800E8103
:100480001F819101281B390BB90137FF04C0662772
:100490007727621B730B603271050CF061C0121676
:1004A00013066CF537014801062E04C09694879414
:1004B000779467940A94D2F721E030E040E050E06E
:1004C00004C0220F331F441F551F6A95D2F72150D5
:1004D0003040404050402E213F21402351232115E0
:1004E00031054105510521F021E030E040E050E0C8
:1004F00079018A01E628F728082919293CC0232B0D
:10050000D1F1260E371E35014601062E04C0969401
:100510008794779467940A94D2F721E030E040E022
:1005200050E004C0220F331F441F551F6A95D2F7B5
:1005300021503040404050402A213B214C215D2138
:10054000211531054105510521F021E030E040E061
:1005500050E059016A01A628B728C828D9280BC03D
:10056000821593052CF01C01AA24BB24650103C04D
:10057000EE24FF24870111969C91D20111968C9153
:10058000981709F445C0992339F0A80197012A1951
:100590003B094C095D0906C0A60195012E193F09CA
:1005A000400B510B57FD08C01182338222822483F5
:1005B0003583468357831DC081E081833382228245
:1005C00088279927DC01821B930BA40BB50B84832E
:1005D0009583A683B7830DC0220F331F441F551F79
:1005E0002483358346835783828193810197938344
:1005F00082832481358146815781DA01C9010197BF
:10060000A109B1098F5F9F4FAF4FBF4328F30BC0C4
:10061000918333822282EA0CFB1C0C1D1D1DE48297
:10062000F5820683178383E08083248135814681A8
:10063000578157FF1AC0C901AA2797FDA095BA2F65
:1006400081709070A070B07056954795379527953A
:10065000822B932BA42BB52B84839583A683B783FE
:1006600082819381019693838283DF0101C0D2014D
:10067000CD01CDB7DEB7E2E104C5A0E2B0E0E2E42F
:10068000F3E0EFC469837A838B839C832D833E835D
:100690004F835887E9E0EE2EF12CEC0EFD1ECE01C3
:1006A0000196B701EDD38E010F5E1F4FCE01059667
:1006B000B801E6D38A8991E089278A8BC701B801FE
:1006C000AE01475E5F4F8FDE06D3A096E6E0E5C43D
:1006D000A0E2B0E0EDE6F3E0C4C469837A838B83E3
:1006E0009C832D833E834F835887F9E0EF2EF12CB6
:1006F000EC0EFD1ECE010196B701C2D38E010F5E36
:100700001F4FCE010596B801BBD3C701B801AE019A
:10071000475E5F4F68DEDFD2A096E6E0BEC4A0E28F
:10072000B0E0E4E9F3E091C469837A838B839C832E
:100730002D833E834F835887CE010196BE01675FAC
:100740007F4F9ED3CE010596BE016F5E7F4F98D33B
:100750009985923088F089898230C8F0943019F4F4
:10076000823051F404C0843029F4923081F481E065
:1007700091E0C6C0923049F420E09A858A899813A6
:1007800021E02A87CE010996BBC0823049F420E0DF
:100790009A858A89981321E02A8BCE014196B0C0B0
:1007A0002D843E844F8458886D887E888F88988CED
:1007B000EE24FF248701AA24BB24650140E050E019
:1007C00060E070E0E0E0F0E0C10181709070892BA2
:1007D000E9F0E60CF71C081D191D9A01AB012A0D62
:1007E0003B1D4C1D5D1D80E090E0A0E0B0E0E614F4
:1007F000F7040805190520F481E090E0A0E0B0E0DE
:10080000BA01A901480F591F6A1F7B1FAA0CBB1C04
:10081000CC1CDD1C97FE08C081E090E0A0E0B0E0B9
:10082000A82AB92ACA2ADB2A3196E032F10549F012
:10083000660C771C881C991C56944794379427940F
:10084000C3CFFA85EA892B893C898B859C85280F43
:10085000391F2E5F3F4F17C0CA0181709070892BDE
:1008600061F016950795F794E79480E090E0A0E09A
:10087000B0E8E82AF92A0A2B1B2B7695679557953D
:1008800047952F5F3F4F77FDE7CF0CC0440F551FB3
:10089000661F771F17FD4160EE0CFF1C001F111F24
:1008A00021503040403090E0590790E0690790E4D3
:1008B000790760F32B8F3C8FDB01CA018F77907033
:1008C000A070B07080349105A105B10561F447FDB9
:1008D0000AC0E114F1040105110529F0405C5F4FE5
:1008E0006F4F7F4F40781A8EFE1711F081E08A8F8C
:1008F0004D8F5E8F6F8F78A383E0898FCE014996ED
:10090000EAD1A096E2E1BDC3A8E1B0E0E9E8F4E0F5
:10091000A4C369837A838B839C832D833E834F8317
:100920005887B9E0EB2EF12CEC0EFD1ECE0101969E
:10093000B701A6D28E010F5E1F4FCE010596B801FA
:100940009FD22985223008F47EC03989323010F4D4
:10095000B8017CC08A859A8989278A87243011F05A
:10096000223031F4231709F06EC061E071E06EC0EF
:10097000343039F41D861E861F86188A1C861B8615
:1009800004C0323021F484E08987B7015FC02B8531
:100990003C858B899C89281B390B3C872B87ED84F0
:1009A000FE840F851889AD88BE88CF88D88CEA145C
:1009B000FB040C051D0540F4EE0CFF1C001F111F6D
:1009C000215030403C872B8720E030E040E050E071
:1009D00080E090E0A0E0B0E460E070E0EA14FB04A6
:1009E0000C051D0540F0282B392B4A2B5B2BEA18F0
:1009F000FB080C091D09B695A79597958795EE0CF0
:100A0000FF1C001F111F6F5F7F4F6F31710531F7A2
:100A1000DA01C9018F779070A070B07080349105B1
:100A2000A105B10561F427FD0AC0E114F104010537
:100A3000110529F0205C3F4F4F4F5F4F20782D87E5
:100A40003E874F87588BBE01675F7F4FCB0143D1F5
:100A50006896EAE01EC3A8E1B0E0E0E3F5E001C378
:100A600069837A838B839C832D833E834F8358874E
:100A700089E0E82EF12CEC0EFD1ECE010196B701A7
:100A8000FFD18E010F5E1F4FCE010596B801F8D140
:100A90008985823038F08989823020F0C701B80119
:100AA00067D201C08FEF6896E6E0F7C2ACE0B0E035
:100AB000EBE5F5E0DAC269837A838B839C83CE0110
:100AC0000196BE016B5F7F4FDBD18D81823061F17A
:100AD000823050F1843021F48E81882351F12EC070
:100AE0002F81388537FD20C06E812F3131051CF0F4
:100AF0006623F9F023C08EE190E0821B930B2985D9
:100B00003A854B855C8504C0569547953795279562
:100B10008A95D2F76623B1F050954095309521958E
:100B20003F4F4F4F5F4F0EC020E030E040E050E0BD
:100B300009C02FEF3FEF4FEF5FE704C020E030E048
:100B400040E050E8B901CA012C96E2E0AAC2A8E050
:100B5000B0E0ECEAF5E081C27B018C016115710522
:100B60008105910519F482E089835FC083E0898360
:100B70008EE1C82ED12CDC82CB82ED82FE820F83E7
:100B80001887C801B70158D0FC013197F7FF3BC067
:100B9000222733272E1B3F0B57016801022E04C06A
:100BA000D694C794B794A7940A94D2F740E050E043
:100BB00060E070E081E090E0A0E0B0E004C0880F69
:100BC000991FAA1FBB1F2A95D2F70197A109B10946
:100BD0008E219F21A023B1230097A105B10521F00B
:100BE00041E050E060E070E04A295B296C297D29F2
:100BF0004D835E836F8378878EE190E08E1B9F0B21
:100C00009C838B8312C0309781F00E2E04C0EE0CB3
:100C1000FF1C001F111F0A94D2F7ED82FE820F8382
:100C20001887CE1ADF0ADC82CB821A82CE010196A7
:100C300052D02896EAE02DC2EF92FF920F931F93B5
:100C40007B018C0180E0E81680E0F80681E008076F
:100C500080E0180788F48FEFE816F104010511050C
:100C600031F028F088E090E0A0E0B0E017C080E02C
:100C700090E0A0E0B0E012C080E0E81680E0F80666
:100C800080E0080781E0180728F088E190E0A0E004
:100C9000B0E004C080E190E0A0E0B0E020E230E00D
:100CA00040E050E0281B390B4A0B5B0B04C0169543
:100CB0000795F794E7948A95D2F7F701E75FFE4F1F
:100CC0008081281B310941095109C9011F910F91E8
:100CD000FF90EF900895DF92EF92FF920F931F9392
:100CE000FC01E480F58006811781D180808182300B
:100CF00048F480E090E0A0E1B0E0E82AF92A0A2B6D
:100D00001B2BA5C0843009F49FC0823021F4EE244F
:100D1000FF24870105C0E114F1040105110519F450
:100D2000E0E0F0E096C0628173819FEF623879075E
:100D30000CF05BC022E83FEF261B370B2A31310550
:100D40002CF020E030E040E050E02AC0B801A701DC
:100D5000022E04C076956795579547950A94D2F769
:100D600081E090E0A0E0B0E004C0880F991FAA1FC6
:100D7000BB1F2A95D2F70197A109B1098E219F21A6
:100D8000A023B1230097A105B10521F081E090E0F7
:100D9000A0E0B0E09A01AB01282B392B4A2B5B2B4A
:100DA000DA01C9018F779070A070B070803491051E
:100DB000A105B10539F427FF09C0205C3F4F4F4F13
:100DC0005F4F04C0215C3F4F4F4F5F4FE0E0F0E0CA
:100DD0002030A0E03A07A0E04A07A0E45A0710F04C
:100DE000E1E0F0E079018A0127C06038710564F51F
:100DF000FB01E158FF4FD801C7018F779070A070B9
:100E0000B07080349105A105B10539F4E7FE0DC03D
:100E100080E490E0A0E0B0E004C08FE390E0A0E0C8
:100E2000B0E0E80EF91E0A1F1B1F17FF05C016953C
:100E30000795F794E794319687E016950795F79410
:100E4000E7948A95D1F705C0EE24FF248701EFEFE0
:100E5000F0E06E2F679566276795902F9F77D79460
:100E6000DD24D7948E2F8695492F462B582F5D2948
:100E7000B701CA011F910F91FF90EF90DF90089585
:100E8000FC01DB01408151812281622F6F7770E08C
:100E9000221F2227221F9381892F880F822B282F20
:100EA00030E0991F9927991F11969C93119721154E
:100EB0003105A9F5411551056105710511F482E06F
:100EC00037C082E89FEF13969C938E9312979A01F6
:100ED000AB0167E0220F331F441F551F6A95D1F7FE
:100EE00083E08C930DC0220F331F441F551F1296B1
:100EF0008D919C911397019713969C938E931297C3
:100F0000203080E0380780E0480780E4580758F335
:100F100014962D933D934D935C93179708952F3F0F
:100F2000310579F4411551056105710519F484E025
:100F30008C93089564FF03C081E08C9312C01C92CF
:100F400010C02F57304013963C932E93129783E096
:100F50008C9387E0440F551F661F771F8A95D1F742
:100F6000706414964D935D936D937C9317970895D9
:100F70001F93DC01FB019C91923008F447C08081F3
:100F8000823008F443C0943051F411961C9184309F
:100F900099F58181682F70E0611B71093FC0843031
:100FA00021F0923031F48230B9F18181882389F1C6
:100FB0002DC011961C9111978230F1F08181181784
:100FC000D9F412962D913C911397828193818217C7
:100FD000930794F028173907BCF014968D919D91D2
:100FE0000D90BC91A02D2481358146815781281711
:100FF00039074A075B0718F4112341F00AC082172A
:101000009307A407B50740F4112319F061E070E0DD
:1010100005C06FEF7FEF02C060E070E0CB011F9171
:101020000895AA1BBB1B51E107C0AA1FBB1FA6172F
:10103000B70710F0A61BB70B881F991F5A95A9F781
:1010400080959095BC01CD0108952F923F924F92CB
:101050005F926F927F928F929F92AF92BF92CF9248
:10106000DF92EF92FF920F931F93CF93DF93CDB751
:10107000DEB7CA1BDB0B0FB6F894DEBF0FBECDBFC9
:1010800009942A88398848885F846E847D848C849A
:101090009B84AA84B984C884DF80EE80FD800C81A3
:1010A0001B81AA81B981CE0FD11D0FB6F894DEBF86
:0C10B0000FBECDBFED010895F894FFCFF6
:00000001FF
